:100000000C9452030C946D030C946D030C946D03CB
:100010000C946D030C946D030C946D030C946D03A0
:100020000C946D030C946D030C946D030C946D0390
:100030000C946D030C94DB160C946D030C94131745
:100040000C946D030C946D030C946D030C946D0370
:100050000C946D03547970652061736D20736F7516
:100060007263650053617665202573202E2E2E0065
:10007000426C6F636B3A2530327800446F6E6500D6
:1000800043616E6E6F74206F70656E2046696C659B
:1000900020257321005A752077656E6967205061AD
:1000A00072616D6574657221004C6F616420257307
:1000B0002000253034782025303478002025303455
:1000C0007800202E2E2E00426C6F636B3A25303262
:1000D0007800446F6E650A000D4346580D002D20D0
:1000E0004E6F204B432D42696E617279000D0842BC
:1000F0006F6F74206572726F72210046696C6520A3
:100100006E6F7420666F756E64000D08426F6F74B9
:1001100066696C65206E6F74206578697374210060
:1001200053657269616C3C2D3E434620302E303160
:100130000A006B65696E652043462D4B61727465DC
:10014000203F0A000D0843462D4B61727465206EF6
:10015000696368742065726B616E6E7421000A4376
:10016000463E0053657269616C3C2D3E434620302B
:100170002E30310A0052656164790A000A437572B3
:1001800072656E7420536563746F7220256C750AF6
:10019000000A43757272656E7420436C75737465E2
:1001A0007220256C7520536563746F7220256C7501
:1001B0000A0053746174757362797465206669729C
:1001C000737420506172746974696F6E3A200030E4
:1001D0007830303D4E6F20426F6F74706172746979
:1001E00074696F6E0A00307838303D426F6F7470FA
:1001F0006172746974696F6E0A0050617274697417
:10020000696F6E20547970653A20004E6F742075C6
:100210007365640A00444F532031322D62697420A3
:100220004641540A00444F532031362D62697420F0
:100230003C33324D0A00457874656E6465640A008B
:10024000444F532031362D626974203E3D33324D88
:100250000A0057696E39352046415433320A005737
:10026000696E393520464154333220284C424129A9
:100270000A0057696E39352046415431360A005715
:10028000696E393520464154313620284C42412987
:100290000A0057696E393520457874656E64656467
:1002A0000A00556E6B6E6F776E0A00426F6F747343
:1002B0006563746F723A20256C750A005365637428
:1002C0006F72732070657220436C75737465723A37
:1002D0002025750A00526573657276656420536542
:1002E00063746F72733A2025750A004E756D6265EE
:1002F00072206F662046415427733A2025750A0004
:10030000536563746F727320706572204641543A6E
:1003100020256C750A00546F74616C2053656374FA
:100320006F727320283136426974293A202575206E
:1003300020283332426974293A20256C750A00520C
:100340006F6F7444697220456E74727927733A2016
:1003500025750A00466972737420526F6F74446980
:1003600072536563746F723A20256C750A00466992
:100370007273742044617461536563746F723A20C0
:10038000256C750A004461746120536563746F7253
:1003900073206F6620506172746974696F6E3A20C1
:1003A000256C750A004461746120436C7573746533
:1003B0007273206F6620506172746974696F6E3A4F
:1003C00020256C750A0046697273742046415420DA
:1003D000536563746F723A20256C750A0054797006
:1003E00065206F66204641543A2046415425750ADF
:1003F00000426F6F74736563746F72204F454D2DAB
:100400004E414D453A20000A566F6C756D65204C83
:100410006162656C3A20000A46696C652053797305
:1004200074656D20537472696E673A20000A000A81
:10043000004472697665204E616D653A20000A00BD
:100440005265766973696F6E3A20000A5365726966
:10045000616C4E756D6265723A20000A432F482F19
:100460005320256C752F25752F256C750A00436167
:100470007061636974793A20256C756B420A005388
:10048000657269616C20436F6D7061637420466CA6
:10049000617368204F532056302E30310A0A287776
:1004A00029323030342062792041726E65204669ED
:1004B000747A656E7265697465720A5765623A206E
:1004C0007777772E6669747A656E7265697465727E
:1004D0002E64650A0A54687820746F20486F6C6730
:1004E0006572204B6C6162756E646520666F722068
:1004F00068697320776F726B0A004563686F206FBD
:100500006E0A0042696E617279206F66660A004663
:1005100072656520436C75737465723A20256C753D
:100520002030782530386C780A00446972206E6F6C
:100530007420666F756E6400536563746F72206E0D
:10054000756D62657220256C7520746F6F2062690D
:10055000670A004572726F72000A436F6D6D616EBB
:1005600064204C6973743A0A00482020202020201F
:1005700020202073686F7720746869732068656C29
:10058000700A005620202020202020202073686F31
:10059000772076657273696F6E20696E666F0A00E8
:1005A00049202020202020202020647269766520A8
:1005B000696E666F726D6174696F6E730A005220A6
:1005C00020202020202020206368616E6765207431
:1005D0006F20726F6F74206469726563746F7279D3
:1005E0000A00442020202020202020206C697374E1
:1005F0002063757272656E74206469726563746FCE
:1006000072790A00434420286E616D652920636871
:10061000616E67652064697220286E616D65290AC4
:10062000004C20286E616D652920206C6F6164206C
:1006300066696C6520286E616D65290A0A00532081
:1006400041414141204545454520535353532028BE
:100650006E616D65290A00202073617665206669E8
:100660006C6520286E616D652920535353533D46B8
:10067000464646206E6F206175746F0A004C20005C
:100680000A000A5620000A4420000A462000203CA6
:10069000564F4C3E00203C4449523E002025203914
:1006A0006C75000011241FBECFE5D8E0DEBFCDBFC2
:1006B00010E0A0E6B0E0E4EEF3E402C005900D9295
:1006C000A43CB107D9F715E0A4ECB0E001C01D923D
:1006D000A73FB107E1F70C940E070C940000EF92CE
:1006E000FF920F931F93CF93DF9361E080E690E03A
:1006F0000E94AB128823A1F10E94C50884E590E016
:100700009F938F930E9401208DE00E943F170F90CE
:100710000F901BC0C0E0D0E0822F9927C817D907DF
:10072000A0F47C018E010C531F4FF80180810E94C0
:100730003F17F80180818D3021F484EF91E00E9411
:1007400061082196CE15DF0568F360E870E084EC5F
:1007500090E00E94A011282F8823E1F60E94F21356
:10076000DF91CF911F910F91FF90EF900895FC01C1
:1007700020E030E040E050E070E06191862F80534F
:100780008A3098F4689413F8220F331F441F551FC2
:100790001694D1F7862F9927C097AA2797FDA09581
:1007A000BA2F280F391F4A1F5B1F862F81548630AE
:1007B00098F4689413F8220F331F441F551F1694A2
:1007C000D1F7862F9927C797AA2797FDA095BA2F0B
:1007D000280F391F4A1F5B1F7F5F743070F2CA01F8
:1007E000B90108954F925F926F927F928F929F927C
:1007F000AF92BF92CF92DF92EF92FF920F931F932F
:10080000CF93DF93CDB7DEB72D970FB6F894DEBF49
:100810000FBECDBF6C010E945D21409708F4A0C1BE
:10082000C6010E94B703DC01CB014C01C60105964D
:100830000E94B703DC01CB013C01C6010A960E946D
:10084000B703DC01CB012C01AA24BB247501CE0126
:10085000019620E2F701E80FF91F20830894E11CBC
:10086000F11C3DE0E316F104A8F3EE24FF249E0101
:100870002F5F3F4FF601EE0DFF1D86858E3231F45E
:100880000F2EF9E0AF2EBB24F02D0DC0A501420FB5
:10089000531FD601AE0DBF1D1E968C91FA018083A9
:1008A0000894A11CB11CFDE0AF16B10428F00F2E76
:1008B000F4E1EF2EFF24F02D0894E11CF11C8DE0F3
:1008C000E816F104B8F20E94C508FF246894F1F814
:1008D000F09248018601015F1F4F1F930F9384E63A
:1008E00090E09F938F930E9401206F2DC8010E947A
:1008F000AB120F900F900F900F90882309F41CC13A
:1009000083EC8093C4008BE48093C50083E48093E0
:10091000C6008DE28093C70084E58093C80021E47F
:100920002093C90080E58093CA0085E48093CB00C2
:1009300090E29093CC0082E68093CD0089E780938B
:10094000CE009093CF002093D00086E48093D10016
:100950008EE28093D2009093D30081E08093D40004
:1009600061E170E084EC90E00E948510EE24FF24A9
:1009700084EC90E0F701E80FF91F10820894E11C65
:10098000F11CE2E8EE16F104A8F3FFEF4F16FFEFBB
:100990005F0611F462E001C063E0EE24FF2444EC42
:1009A00050E09E012F5F3F4FC701840F951FDC0170
:1009B0001197F701E20FF31F80818C930894E11CDB
:1009C000F11C8CE0E816F10478F36093D400809277
:1009D000D500892D99278093D6006092D700872D66
:1009E00099278093D800633031F44092D900852D47
:1009F00099278093DA0060E870E084EC90E00E9430
:100A000085105301A818B9080894A11CB11C8BE1EA
:100A10000E943F1781E090E00E94610886E50E94F5
:100A20003F17882D0E943F17892D99270E943F1755
:100A30008A2D0E943F170E9466178B2D99270E94CE
:100A40003F1761E082E00E94AF08EE24FF2484ECAF
:100A500090E0F701E80FF91F10820894E11CF11CE7
:100A6000E2E8EE16F104A8F399249394EE24FF240F
:100A7000A114B10409F44CC00F2EF4ECCF2EF0E019
:100A8000DF2EF02D892C0894E11CF11C87010C0D40
:100A90001D1D0E942017F80180830894A108B10849
:100AA000F0E8EF16F10480F1929A93949092C400CA
:100AB00080924801682D82E00E94AF088091C400B6
:100AC00099279F938F9380E790E09F938F930E9445
:100AD000012061E870E0C6010E948510EE24FF2429
:100AE0000F900F900F900F9084EC90E0F701E80FBB
:100AF000F91F10820894E11CF11C22E8E216F104AF
:100B0000A8F3EE24FF249298A114B10409F0BBCFFE
:100B10008FEF8093C40061E870E084EC90E00E9465
:100B20008510109248018BE790E09F938F930E946D
:100B300001200E94F2131CC010924801F601878523
:100B4000992787FD90959F938F9380E890E09F93DE
:100B50008F930E9401200F900F900F900F900AC06A
:100B60001092480185E990E09F938F930E940120A5
:100B70000F900F902D960FB6F894DEBF0FBECDBF2D
:100B8000DF91CF911F910F91FF90EF90DF90CF9069
:100B9000BF90AF909F908F907F906F905F904F909D
:100BA0000895AF92BF92CF92DF92EF92FF920F9390
:100BB0001F93CF93DF93EC0161E00E94AB12882377
:100BC00009F410C10E94C50882E080934801DF93B8
:100BD000CF9389EA90E09F938F930E940120109217
:100BE000480160E170E084EC90E00E94A01161E0B7
:100BF00070E084EC90E00E94A01160E870E084EC6A
:100C000090E00E94A011C090D4008C2D82500F90D3
:100C10000F900F900F90823008F0D8C02091D5002F
:100C20008091D600992787FD9095982F8827EC0111
:100C3000C20FD11D2091D7008091D800992787FD40
:100C40009095982F88278C01020F111D2091D900B3
:100C50008091DA00992787FD9095982F88275C016D
:100C6000A20EB11C80914601882391F01F930F932F
:100C7000DF93CF9382EB90E09F938F930E940120AC
:100C80008DB79EB706960FB6F8949EBF0FBE8DBF68
:100C900093E0C91681F480914601882361F0BF92E8
:100CA000AF928CEB90E09F938F930E9401200F9066
:100CB0000F900F900F9080914601882341F082ECB5
:100CC00090E09F938F930E9401200F900F907801E6
:100CD000EC1AFD0A0894E11CF11C8BE10E943F17FD
:100CE00081E090E00E94610884E50E943F178C2F0C
:100CF0000E943F178D2F99270E943F178E2D0E942B
:100D00003F178F2D99270E943F17DD24D3942BC0C6
:100D1000D09248016D2D82E00E94AF088091C400FE
:100D200099279F938F9387EC90E09F938F930E94D6
:100D300001200F900F900F900F90C1E0D0E0123083
:100D400090F0012F1127E114F10449F0FE01EC535A
:100D5000FF4F80810E943F170894E108F108219617
:100D6000C017D10780F361E870E084EC90E00E9446
:100D7000A011182F882361F6109248018091460136
:100D8000882319F082ED90E002C088ED90E09F93F7
:100D90008F930E9401200F900F9081E090E00E94BD
:100DA000610883E0C81679F58BE10E943F1781E066
:100DB00090E00E94610885E50E943F178A2D0E94FD
:100DC0003F178B2D99270E943F171DC01092480195
:100DD00080914601882319F08EED90E00EC08DEED3
:100DE00090E00BC01092480180914601882319F0D1
:100DF0008BEF90E002C08AE091E09F938F930E9476
:100E000001200F900F90DF91CF911F910F91FF90D4
:100E1000EF90DF90CF90BF90AF900895CFE5D8E0EE
:100E2000DEBFCDBF9FEF94BB15BA86EF81BB8AE0D2
:100E300082BB1ABA9BBB97BB98BB80B710BE60EB56
:100E400074E080E090E00E946D17929A78940E947E
:100E5000CF0811E0109348010E94C50880E291E09C
:100E60009F938F930E940120612F82E00E94AF0820
:100E700080E00E94DC0C0F900F908117A1F082E3BC
:100E800091E09F938F930E94012082E0809348011C
:100E90000F900F9084E491E09F938F930E94012024
:100EA0000F900F90FFCF0E943F10109246011092BA
:100EB00047018DE690E00E94D10584E690E00E9413
:100EC000610881E080934601929A6CED75ED80E0B7
:100ED00090E00E946D1792980E94661711E0809131
:100EE0004601813021F48EE591E00E94ED1F1093C0
:100EF00048010E94C50883E691E09F938F930E946A
:100F00000120612F82E00E94AF080F900F9085E7CB
:100F100091E09F938F930E940120109248010E94BC
:100F2000A9170F900F9099278530910509F440C0BB
:100F3000863091056CF48230910509F459C08330F4
:100F400091051CF40197A1F0CACF0497A1F0C7CF77
:100F50008730910509F47FC0873091050CF44EC0AD
:100F60008830910509F4A3C0099709F4A5C0B7CF4B
:100F70000E944E1AB4CF80915D01803249F01092E8
:100F80004D0110924E0110924F011092500110C06D
:100F900080919A0190919B01A0919C01B0919D013B
:100FA00080934D0190934E01A0934F01B093500157
:100FB00080914D0190914E01A0914F01B09150014F
:100FC0000097A105B10529F480E090E00E941C1F64
:100FD00086CF80914D0190914E01A0914F01B0912B
:100FE000500140E050E0BC01CD010E94B11E77CF1E
:100FF00081E00E94DC0C0E943F1071CF8091620161
:1010000090916301A0916401B091650143EB53E0BD
:10101000BC01CD010E94C61483EB93E00E948614AC
:1010200080914601882309F45ACF80916201909102
:101030006301A0916401B0916501BF93AF939F9349
:101040008F938CE791E09F938F930E9401208DB73F
:101050009EB7069626C080914601882309F43FCFAB
:101060008091620190916301A0916401B09165014A
:10107000BF93AF939F938F9380917C0190917D015B
:10108000A0917E01B0917F01BF93AF939F938F9307
:1010900081E991E09F938F930E9401208DB79EB7C5
:1010A0000A960FB6F8949EBF0FBE8DBF18CF86EC80
:1010B00090E00E94D10513CF86EC90E00E94F203ED
:1010C0000ECF0F931F93CF93DF938C01C0E0D0E03E
:1010D000C817D90738F48AE00E9477082196C0170C
:1010E000D107C8F3DF91CF911F910F91089520E0B0
:1010F0002817D8F490E00000000000000000000075
:1011000000000000000000000000000000000000DF
:1011100000000000000000000000000000009F5FD1
:10112000983248F32F5F281728F30895949885BBC9
:10113000949A949881E00E9477080895CF93DF9362
:10114000EC018881882341F02196882329F00E94B0
:10115000960888818823C1F7DF91CF9108959598EB
:1011600099278130910519F0029721F006C0862F4A
:10117000815804C0862F815401C080E80E949608DF
:10118000959A81E00E9477080895959881E00E94E1
:101190009608959A85E090E00E94610808951F9353
:1011A000CF93DF93959894988FEF90E00E94610819
:1011B000C0E0D0E010E315BB949A94988AE090E0E8
:1011C0000E9461082196C330D105ACF388E30E94E8
:1011D000960885E090E00E94610884E10E949608EC
:1011E00085E090E00E9461088CE00E94960885E00E
:1011F00090E00E94610886E00E94960885E090E0F9
:101200000E94610882E00E94960885E090E00E94BA
:101210006108959ADF91CF911F910895CF93C82FC0
:1012200082958F708A3010F4805D01C0895C0E94C5
:1012300096088C2F8F708A3010F4805D01C0895C15
:101240000E949608CF910895EF92FF920F931F93FB
:101250007B018C01892F9927AA27BB270E940E09A1
:10126000C801AA27BB270E940E09BB27A12F902FD8
:101270008F2D0E940E098E2D0E940E091F910F9135
:10128000FF90EF900895AF92BF92CF92DF92EF92CE
:10129000FF920F931F935B016C010E94A1097B01D8
:1012A0008C018FEFE8168FEFF8068FEF08078FEFAE
:1012B0001807E1F18091690190916A01A0916B0199
:1012C000B0916C018E159F05A007B10778F1A114AC
:1012D000B104C104D10431F0A8019701C601B501E0
:1012E0000E94280A80915D018C3041F42FEF3FE08D
:1012F00040E050E0C801B7010E94280A80915D01DA
:10130000803141F42FEF3FEF40E050E0C801B701DA
:101310000E94280A80915D01803241F42FEF3FEF57
:101320004FEF5FE0C801B7010E94280AC801B7016A
:101330001F910F91FF90EF90DF90CF90BF90AF90F3
:101340000895AF92BF92CF92DF92EF92FF920F93E8
:101350001F935B016C017B018C010894E11CF11C63
:10136000011D111D8091690190916A01A0916B018D
:10137000B0916C01E816F9060A071B07E0F4C801F2
:10138000B7010E949C0BDC01CB010097A105B105C0
:1013900091F00894E11CF11C011D111D809169015F
:1013A00090916A01A0916B01B0916C01E816F90669
:1013B0000A071B0720F38091690190916A01A091AF
:1013C0006B01B0916C01E816F9060A071B0718F1CA
:1013D000EE24FF2487016894E1F8AE14BF04C00630
:1013E000D106A0F0C801B7010E949C0BDC01CB0123
:1013F0000097A105B10551F00894E11CF11C011DF5
:10140000111DAE14BF04C006D10660F7EA14FB0438
:101410000C051D0568F48091690190916A01A09105
:101420006B01B0916C01E816F9060A071B0728F05A
:101430006FEF7FEF8FEF9FEF02C0C801B7011F91E1
:101440000F91FF90EF90DF90CF90BF90AF900895F5
:101450002F923F924F925F926F927F928F929F92C4
:10146000AF92BF92CF92DF92EF92FF920F931F93B2
:10147000CF93DF935B016C0139014A0180916901CF
:1014800090916A01A0916B01B0916C01A816B90608
:10149000CA06DB0608F03BC180915D018C3009F083
:1014A000A4C0D601C501880F991FAA1FBB1F8A0DB2
:1014B0009B1DAC1DBD1DB695A795979587959C0165
:1014C000AD01317040705070E9019C01AD01012EF9
:1014D00019E056954795379527951A95D1F7102D10
:1014E0008091590190915A01A0915B01B0915C01EA
:1014F00019012A01280E391E4A1E5B1E9301D601CE
:10150000C50181709070A070B070892B31F0229568
:101510003295307F3227207F3227E22E832F992782
:10152000182F43EB53E0C201B1010E94C61481E0C1
:10153000CF3FD807F1F5E2EBF5E0D601C5018170A8
:101540009070A070B070892B39F08091B2058F70C7
:101550008E298093B20501C0E08243EB53E0C201C3
:10156000B1010E942F15D201C1010196A11DB11D2B
:1015700043EB53E0BC01CD010E94C614E3EBF3E062
:10158000D601C50181709070A070B070892B19F0E0
:101590001093B30304C08081807F812B8083D201AC
:1015A000C1010196A11DB11D43EB53E0BC01CD016A
:1015B0001AC0FE01ED54FC4FD601C5018170907038
:1015C000A070B070892B31F080818F708E2981934B
:1015D000108305C0E1928081807F812B808343EB63
:1015E00053E0C201B1010E942F1580915D0180314D
:1015F000D1F586017501EA0CFB1C0C1D1D1DA8010F
:101600009701012E19E056954795379527951A951C
:10161000D1F7102D8091590190915A01A0915B0151
:10162000B0915C0119012A01280E391E4A1E5B1E69
:1016300043EB53E0C201B1010E94C614D801C701B7
:101640009170A070B07023EB33E0FC01E20FF31F48
:101650006192BB27A92D982D872D8083A901C201F6
:10166000B1010E942F1580915D01803209F04FC0B9
:1016700086017501EE0CFF1C001F111FEE0CFF1CF4
:10168000001F111FA8019701012E19E056954795DB
:10169000379527951A95D1F7102D80915901909182
:1016A0005A01A0915B01B0915C0119012A01280E39
:1016B000391E4A1E5B1E43EB53E0C201B1010E947A
:1016C000C614D801C7019170A070B07023EB33E04D
:1016D000FC01E20FF31F8FEF9FEFAFEFBFE0682237
:1016E00079228A229B226192BB27A92D982D872DD2
:1016F0008193C401AA27BB278193892D9927AA2703
:10170000BB278083A901C201B1010E942F1580E08F
:1017100090E0DF91CF911F910F91FF90EF90DF90BC
:10172000CF90BF90AF909F908F907F906F905F9081
:101730004F903F902F9008958F929F92AF92BF92BB
:10174000CF92DF92EF92FF920F931F93CF93DF938D
:101750006B017C018091690190916A01A0916B01FC
:10176000B0916C01C816D906EA06FB0608F0EDC078
:1017700080915D018C3009F074C0D701C601880FDB
:10178000991FAA1FBB1F8C0D9D1DAE1DBF1DB695B9
:10179000A795979587959C01AD0131704070507069
:1017A000E9014C015D01072E79E0B694A794979466
:1017B00087947A95D1F7702D8091590190915A01B3
:1017C000A0915B01B0915C01880D991DAA1DBB1D04
:1017D00043EB53E0BC01CD010E94C61421E0CF3F92
:1017E000D20731F502EB15E08091B205C82FDD2755
:1017F0008091590190915A01A0915B01B0915C01D7
:10180000880D991DAA1DBB1D0196A11DB11DA80122
:101810004F5F5140BC01CD010E94C614F801EF5F3B
:10182000F14080819927982F8827C80FD91F05C0BC
:10183000FE01ED54FC4FC081D181D701C6018170FA
:101840009070A070B070892B39F0D295C295CF708E
:10185000CD27DF70CD2701C0DF70BE018827992713
:1018600078C080915D018031A9F5D701C6018C0D4A
:101870009D1DAE1DBF1D7C018D019C01AD01012E82
:1018800019E056954795379527951A95D1F7102D5C
:101890008091590190915A01A0915B01B0915C0136
:1018A000820F931FA41FB51F43EB53E0BC01CD0172
:1018B0000E94C614D801C7019170A070B070FC01DD
:1018C000ED54FC4F808191819C0144275527CA012A
:1018D000B9013FC080915D018032B9F58701760181
:1018E000EE0CFF1C001F111FEE0CFF1C001F111F30
:1018F000A8019701012E19E0569547953795279530
:101900001A95D1F7102D8091590190915A01A0910B
:101910005B01B0915C01820F931FA41FB51F43EBC5
:1019200053E0BC01CD010E94C614D801C7019170DB
:10193000A070B070FC01ED54FC4F80819181A281B8
:10194000B381BC01CD019F7004C06FEF7FEF8FEFBB
:101950009FEFDF91CF911F910F91FF90EF90DF905C
:10196000CF90BF90AF909F908F900895CF93DF93CB
:10197000DC01CB01FD01EC012297E109F109809125
:101980007A01282F332744275527BE01CF010E9413
:101990008321FC01EB0180915E0190915F01A09198
:1019A0006001B0916101C80FD91FEA1FFB1FBE0182
:1019B000CF01DF91CF9108957F928F929F92AF9246
:1019C000BF92CF92DF92EF92FF920F931F93CF932C
:1019D000DF93782E0E949915882309F038C343EBD2
:1019E00053E060E070E080E090E00E94C614C3EB3A
:1019F000D3E0E0907905F0907A0500917B05109195
:101A00007C05772009F48EC082EB91E09F938F9341
:101A10000E9401200F900F9080917105882341F45E
:101A20008FEC91E09F938F930E9401200F900F9075
:101A3000FE01E254FE4F8081803841F486EE91E051
:101A40009F938F930E9401200F900F908AEF91E057
:101A50009F938F930E9401200F900F90FE01EE53F1
:101A6000FE4F808199278630910581F1873091055D
:101A70007CF48130910509F1823091051CF4892BA9
:101A8000C9F036C084309105D9F00597E1F030C037
:101A90008D30910521F18E30910534F48B30910514
:101AA000C1F00C97C9F024C08E309105D9F00F9782
:101AB000E1F01EC08BE092E01DC085E192E01AC00B
:101AC00085E292E017C086E392E014C080E492E0E1
:101AD00011C082E592E00EC08FE592E00BC082E774
:101AE00092E008C08FE792E005C082E992E002C070
:101AF00082EA92E09F938F930E9401200F900F90B3
:101B00001F930F93FF92EF928BEA92E09F938F9334
:101B10000E9401208DB79EB706960FB6F8949EBF1F
:101B20000FBE8DBF43EB53E0C801B7010E94C6143E
:101B30000F2EF3EB8F2EF3E09F2EF02D8091C0033C
:101B400080937A018091C4039091C50390938101A1
:101B5000809380018091C9039091CA03009719F086
:101B6000AA27BB2705C0F40184A195A1A6A1B7A10E
:101B700080936E0190936F01A0937001B0937101F7
:101B8000772009F472C080917A0199279F938F93EF
:101B90008CEB92E09F938F930E9401200F900F9007
:101BA0000F900F90F401868597859F938F9385ED15
:101BB00092E09F938F930E9401200F900F900F90BF
:101BC0000F90F401808999279F938F938BEE92E079
:101BD0009F938F930E9401200F900F900F900F9072
:101BE00080916E0190916F01A0917001B09171018F
:101BF000BF93AF939F938F9380E093E09F938F93D6
:101C00000E9401208DB79EB706960FB6F8949EBF2E
:101C10000FBE8DBFF40180A191A1A2A1B3A1BF937A
:101C2000AF939F938F93838994899F938F9386E13A
:101C300093E09F938F930E9401208DB79EB70896E3
:101C40000FB6F8949EBF0FBE8DBF8091800190911A
:101C500081019F938F938FE393E09F938F930E94D3
:101C600001200F900F900F900F9080918001909124
:101C70008101880F991F82959295907F9827807F88
:101C8000982781509E4F892F992786955C01CC24F7
:101C9000DD24A0929201B0929301C0929401D0925F
:101CA0009501F40186859785AA27BB27E80EF91EC2
:101CB0000A1F1B1FE0925901F0925A0100935B0129
:101CC00010935C0180899927AA27BB2720916E0178
:101CD00030916F014091700150917101BC01CD01B3
:101CE0000E948321DC01CB018E0D9F1DA01FB11F1F
:101CF0008093960190939701A0939801B0939901D6
:101D00008A0D9B1DAC1DBD1D80935E0190935F01EC
:101D1000A0936001B0936101F401838994890097D5
:101D200021F05C01CC24DD2405C0F401A0A0B1A009
:101D3000C2A0D3A0F401868597857C0100271127D6
:101D400080899927AA27BB2720916E0130916F01C6
:101D50004091700150917101BC01CD010E9483211D
:101D6000DC01CB01A8019701280F391F4A1F5B1F17
:101D70008091920190919301A0919401B09195016D
:101D8000820F931FA41FB51FA81AB90ACA0ADB0A3B
:101D900080917A01282F332744275527C601B501A2
:101DA0000E94A221DA01C90120938A0130938B019C
:101DB00040938C0150938D012E5F3F4F4F4F5F4FEB
:101DC0002093690130936A0140936B0150936C0139
:101DD000855F9F40A040B04040F48CE080935D015F
:101DE00088EF9FE0A0E0B0E014C080918A0190915C
:101DF0008B01A0918C01B0918D01855F9F4FA04018
:101E0000B04080F480E180935D0188EF9FEFA0E017
:101E1000B0E080938E0190938F01A0939001B093D6
:101E2000910132C080E280935D0188EF9FEFAFEFB8
:101E3000BFE080938E0190938F01A0939001B093A7
:101E40009101F40184A595A5A6A5B7A580939A0153
:101E500090939B01A0939C01B0939D0180934D01B1
:101E600090934E01A0934F01B0935001BC01CD015E
:101E70000E94B60CDC01CB018093960190939701F0
:101E8000A0939801B0939901772009F4E3C0809161
:101E9000960190919701A0919801B0919901BF93FB
:101EA000AF939F938F9384E593E09F938F930E94CA
:101EB00001208DB79EB706960FB6F8949EBF0FBE51
:101EC0008DBF80915E0190915F01A0916001B09102
:101ED0006101BF93AF939F938F938EE693E09F939F
:101EE0008F930E940120EDB7FEB736960FB6F89497
:101EF000FEBF0FBEEDBFDF92CF92BF92AF9285E8DB
:101F000093E09F938F930E9401208DB79EB7069612
:101F10000FB6F8949EBF0FBE8DBF80918A0190913D
:101F20008B01A0918C01B0918D01BF93AF939F93D2
:101F30008F9385EA93E09F938F930E940120EDB7E2
:101F4000FEB736960FB6F894FEBF0FBEEDBF809178
:101F5000590190915A01A0915B01B0915C01BF932E
:101F6000AF939F938F9386EC93E09F938F930E9400
:101F700001208DB79EB706960FB6F8949EBF0FBE90
:101F80008DBF80915D0199279F938F938DED93E095
:101F90009F938F930E9401200F900F900F900F90AE
:101FA00081EF93E09F938F930E940120C0E00F90F8
:101FB0000F90F401EC0FF11D83810E94D61FCF5FBB
:101FC000C830B8F387E094E09F938F930E9401207C
:101FD000C0E00F900F9080915D01803229F0F401F4
:101FE000EC0FF11D83A507C0C4018C0F911DFC01EE
:101FF000E95BFF4F80810E94D61FCF5FCB3058F343
:1020000087E194E09F938F930E940120C0E00F909E
:102010000F9080915D01803229F0F401EC0FF11DE9
:1020200086A907C0C4018C0F911DFC01EE5AFF4F19
:1020300080810E94D61FCF5FC83058F38DE294E0B4
:102040009F938F930E9401200F900F9003C080E018
:1020500090E007C0772019F084E00E943F1781E0EC
:1020600090E0DF91CF911F910F91FF90EF90DF9063
:10207000CF90BF90AF909F908F907F900895809168
:102080005D01803249F010924D0110924E01109284
:102090004F011092500110C080919A0190919B01C4
:1020A000A0919C01B0919D0180934D0190934E01B0
:1020B000A0934F01B09350011092620110926301FE
:1020C000109264011092650182E090E0A0E0B0E01F
:1020D00080937C0190937D01A0937E01B0937F015A
:1020E0001092720110927301109274011092750196
:1020F0001092820110928301109284011092850146
:1021000010927B0110926D0108954F925F926F9231
:102110007F928F929F92AF92BF92CF92DF92EF9277
:10212000FF920F931F93CF93DF939C012B0180911C
:102130007B01882319F480E090E0F1C03901882404
:102140009924E0908201F090830100918401109124
:1021500085018091490190914A01A0914B01B09174
:102160004C01E81AF90A0A0B1B0B8091A701909108
:10217000A801A091A901B091AA01E816F9060A07E1
:102180001B0708F463C08091860190918701A0919C
:102190008801B09189014FEA51E0BC01CD010E9454
:1021A0002F158091550190915601A0915701B09142
:1021B0005801BC01CD010E944309DC01CB01809391
:1021C000550190935601A0935701B09358018F3F4A
:1021D0002FEF92072FEFA2072FEFB20709F49EC04F
:1021E000BC01CD010E94B60CDC01CB0180935101F2
:1021F00090935201A0935301B093540180938601B0
:1022000090938701A0938801B0938901809149013F
:1022100090914A01A0914B01B0914C012091A701EE
:102220003091A8014091A9015091AA01820F931FFA
:10223000A41FB51F8093490190934A01A0934B01BD
:10224000B0934C01E21AF30A040B150BD801C70135
:10225000072E79E0B695A795979587957A95D1F74A
:10226000702DA82EBB24CC24DD24809151019091A7
:102270005201A0915301B09154018A0D9B1DAC1DD8
:10228000BD1DC0918601D0918701E0918801F09138
:1022900089018C179D07AE07BF07D1F04FEA51E0C7
:1022A000BE01CF010E942F158091510190915201E2
:1022B000A0915301B09154018A0D9B1DAC1DBD1D11
:1022C0008093860190938701A0938801B093890140
:1022D000D801C7019170A070B070FC01E155FE4FAC
:1022E000D3018D913D018083809182019091830182
:1022F000A0918401B09185010196A11DB11D80932B
:10230000820190938301A0938401B0938501089486
:10231000811C911C8414950408F413CFC401DF912F
:10232000CF911F910F91FF90EF90DF90CF90BF90D2
:10233000AF909F908F907F906F905F904F90089597
:102340008F929F92AF92BF92CF92DF92EF92FF92C5
:102350000F931F93CF93DF939C014B0180917B01DF
:10236000882319F480E090E0E9C05901CC24DD24F1
:10237000E0907601F0907701009178011091790159
:102380008091820190918301A0918401B091850197
:10239000E816F9060A071B0708F0CFC0809149012B
:1023A00090914A01A0914B01B0914C01E81AF90AB1
:1023B0000A0B1B0B8091A7019091A801A091A90184
:1023C000B091AA01E816F9060A071B0708F45AC0DB
:1023D0008091550190915601A0915701B0915801FB
:1023E000BC01CD010E949C0BDC01CB018093550107
:1023F00090935601A0935701B0935801BC01CD01B1
:102400000E94B60CDC01CB018093510190935201E4
:10241000A0935301B09354014FEA51E0BC01CD01A8
:102420000E94C6148091510190915201A0915301D4
:10243000B09154018093860190938701A093880105
:10244000B09389018091490190914A01A0914B017B
:10245000B0914C012091A7013091A8014091A901B0
:102460005091AA01820F931FA41FB51F80934901A9
:1024700090934A01A0934B01B0934C01E21AF30AE6
:10248000040B150BD801C701072E79E0B695A79567
:10249000979587957A95D1F7702D282F80915101C6
:1024A00090915201A0915301B0915401FD01EC01B2
:1024B000C20FD11DE11DF11D809186019091870110
:1024C000A0918801B0918901C817D907EA07FB07D5
:1024D00071F0C0938601D0938701E0938801F09357
:1024E00089014FEA51E0BE01CF010E94C614D80114
:1024F000C7019170A070B070FC01E155FE4F808162
:10250000F50181935F018091760190917701A0910F
:102510007801B09179010196A11DB11D80937601DA
:1025200090937701A0937801B09379010894C11C2E
:10253000D11CC814D90408F41BCFC601DF91CF9178
:102540001F910F91FF90EF90DF90CF90BF90AF90D1
:102550009F908F900895EF92FF920F931F93CF93C8
:102560008C01C62F80917A019927982F8827990F7F
:10257000AA2797FDA095BA2F8093A7019093A80151
:10258000A093A901B093AA011092490110924A01A7
:1025900010924B0110924C016130E1F5C8010E948C
:1025A00011148530B9F510927601109277011092CE
:1025B0007801109279018091720190917301A0913C
:1025C0007401B09175018093550190935601A093C9
:1025D0005701B0935801C0937B01BC01CD010E940B
:1025E000B60CDC01CB018093510190935201A09372
:1025F0005301B09354018093860190938701A09377
:102600008801B09389014FEA51E0BC01CD010E94DD
:10261000C614DDC0C23009F0DDC0C8010E9411142B
:10262000853009F097C0E0907201F090730100913D
:1026300074011091750180918E0190918F01A0918C
:102640009001B0919101E816F9060A071B0708F0FE
:1026500045C0C801B7010E949C0B7B018C01809191
:102660008E0190918F01A0919001B0919101E81697
:10267000F9060A071B0720F5E0925501F092560172
:1026800000935701109358018091490190914A019C
:10269000A0914B01B0914C012091A7013091A8016C
:1026A0004091A9015091AA01820F931FA41FB51F49
:1026B0008093490190934A01A0934B01B0934C0140
:1026C00080918E0190918F01A0919001B091910124
:1026D000E816F9060A071B0708F4BBCF2091820110
:1026E000309183014091840150918501809149018D
:1026F00090914A01A0914B01B0914C0179018A015E
:10270000E81AF90A0A0B1B0B8091550190915601AA
:10271000A0915701B0915801BC01CD010E94B60CA7
:102720009B01AC016093510170935201809353015E
:1027300090935401D801C701072E79E0B695A7956B
:10274000979587957A95D1F7702D820F931FA41FC7
:10275000B51F2DC046E651E06EE971E0C8010E9448
:102760006E1F0E94CB1A8823F9F08091720190911C
:102770007301A0917401B0917501809355019093FC
:102780005601A0935701B0935801BC01CD010E949E
:10279000B60CDC01CB018093510190935201A093C0
:1027A0005301B093540103C010927B0113C0809376
:1027B000860190938701A0938801B09389014FEA25
:1027C00051E0BC01CD010E94C614C0937B0181E0A1
:1027D00090E002C080E090E0CF911F910F91FF90B8
:1027E000EF90089580917B01823011F40E94FB13D9
:1027F00010927B01089580917B01882381F0809164
:10280000860190918701A0918801B09189014FEADA
:1028100051E0BC01CD010E942F150E94AD1B08950F
:102820000895AC0180914D0190914E01A0914F010E
:10283000B09150010297A105B10520F4CA010E9490
:102840001C1F0CC080914D0190914E01A0914F0131
:10285000B0915001BC01CD010E94B11E992708958D
:10286000AF92BF92CF92DF92EF92FF920F931F939E
:10287000CF935B016C0180918E0190918F01A091AB
:102880009001B0919101A816B906CA06DB0690F531
:10289000C601B5010E94B60C7B018C01C0E080919D
:1028A0007A01C817A0F44FEA51E0C801B7010E94AD
:1028B000C6148FEA91E00E9486140894E11CF11C72
:1028C000011D111DCF5F80917A01C81760F3C60109
:1028D000B5010E949C0B5B016C0180918E0190916F
:1028E0008F01A0919001B0919101A816B906CA0676
:1028F000DB0670F281E090E0CF911F910F91FF9085
:10290000EF90DF90CF90BF90AF900895EF92FF923D
:102910001F93CF93DF93EC01EE24FF248991109154
:102920004701112319F50E94931780E20E94D61FD8
:10293000C701877090700797D9F480E20E94D61F74
:1029400080E20E94D61FCE01810F911DFC013897B5
:102950008081803208F48EE20E94D61F1F5F1830FB
:1029600090F38FE294E00E94ED1F02C00E943F1797
:102970000894E11CF11C80E0E81682E0F80670F291
:10298000DF91CF911F91FF90EF900895EF92FF920A
:102990000F931F93CF93DF937B018C01EA0180910A
:1029A000AF039091B003A091B103B091B203E816C8
:1029B000F9060A071B0720F40E948A16882319F0DB
:1029C00081E090E045C061E082E00E94C5166E2D76
:1029D00083E00E94C516BB27A12F902F8F2D682F53
:1029E00084E00E94C516C801AA27BB27682F85E08E
:1029F0000E94C516812F9927AA27BB278F70806E4A
:102A0000682F86E00E94C51660E287E00E94C51626
:102A10000E949B16882319F082E090E019C01ABA30
:102A20008FEF8BBB80E00E94D516C49820E030E089
:102A3000C59800000000000089B38993C59A2F5FF4
:102A40003F4F82E02030380798F3C49A80E090E04E
:102A5000DF91CF911F910F91FF90EF900895EF922A
:102A6000FF920F931F93CF93DF937B018C01EA01B9
:102A70008091AF039091B003A091B103B091B203E4
:102A8000E816F9060A071B0720F40E948A16882315
:102A900019F081E090E046C061E082E00E94C51636
:102AA0006E2D83E00E94C516BB27A12F902F8F2D7E
:102AB000682F84E00E94C516C801AA27BB27682F8B
:102AC00085E00E94C516812F9927AA27BB278F7002
:102AD000806E682F86E00E94C51660E387E00E9442
:102AE000C5160E949B16882319F082E090E01AC058
:102AF00080E00E94D5168FEF8ABBC49820E030E0BA
:102B000089918BBBC6980000C69A00002F5F3F4F8B
:102B100082E020303807A0F3C49A1ABA8FEF8BBB3B
:102B200080E090E0DF91CF911F910F91FF90EF90A7
:102B300008958F929F92AF92BF92CF92DF92FF92B1
:102B40000F931F93CF93DF93F82E0E948A1688234A
:102B500019F081E090E0D2C06CEE87E00E94C516CB
:102B60000E949B16882319F082E090E0C7C0C0E065
:102B7000D0E08E010D541C4F80E00E94AC16F8018D
:102B800080832196F2E0C030DF0798F3A090B50370
:102B9000B090B603C090B703D090B8038090B9034B
:102BA0009090BA038091C1039091C203AA27BB27DA
:102BB000AC01332722278091C3039091C403AA2735
:102BC000BB27820F931FA41FB51F8093AF03909361
:102BD000B003A093B103B093B203FF2009F48CC0FB
:102BE00081E394E09F938F930E940120C6E3D0E09D
:102BF0000F900F908E010D541C4FF80181810E949F
:102C0000D61FF80180810E94D61F2296CE35D105AD
:102C100088F38EE394E09F938F930E9401200F909E
:102C20000F9080E494E09F938F930E940120CEE266
:102C3000D0E00F900F908E010D541C4FF801818150
:102C40000E94D61FF80180810E94D61F2296C633AB
:102C5000D10588F38BE494E09F938F930E94012029
:102C6000C4E1D0E00F900F90FE01ED54FC4F808145
:102C70000E94D61F2196C832D105B0F38091AF03D0
:102C80009091B003A091B103B091B203BF93AF9301
:102C90009F938F939F928F92DF92CF92BF92AF922A
:102CA0008BE594E09F938F930E9401208DB79EB790
:102CB0000C960FB6F8949EBF0FBE8DBF8091AF03E8
:102CC0009091B003A091B103B091B203B695A795CE
:102CD00097958795BF93AF939F938F938EE694E0DC
:102CE0009F938F930E940120EDB7FEB736960FB6E3
:102CF000F894FEBF0FBEEDBF80E090E0DF91CF9172
:102D00001F910F91FF90DF90CF90BF90AF909F9059
:102D10008F90089587E00E94AC1680FF03C081E089
:102D200090E0089587E00E94AC16807F8035D1F74F
:102D300080E090E0089587E00E94AC1680FF03C019
:102D400081E090E0089587E00E94AC16887F883586
:102D5000D1F780E090E00895982F1ABA8FEF8BBBDF
:102D6000892F0E94D516C498C59800000000000065
:102D700089B3C59AC49A99270895C59800000000A0
:102D8000000089B3C59A992708951F93162F9FEFC6
:102D90009ABB0E94D5161BBB0000C4980000C698C1
:102DA0000000C69AC49A1F910895982F86B3807F19
:102DB000892B88BB08951F920F920FB60F92112492
:102DC0002F933F934F935F938F939F93EF93FF9333
:102DD0008CB18093B3058091F5058034B8F490915F
:102DE000F6058091F505492F480F512D511D9A0187
:102DF0008F5F8093F505CA01807C9370281B390B87
:102E0000F901EB54FA4F8091B3058083FF91EF9164
:102E10009F918F915F914F913F912F910F900FBE96
:102E20000F901F9018951F920F920FB60F921124BA
:102E300053981092B4050F900FBE0F901F901895E5
:102E40008091F5058823E1F357988091F50581502D
:102E50008093F5052091F60585EB95E0FC01E20FE6
:102E6000F11DE0812F5F2093F6058091F6058034F7
:102E700010F01092F605579A8E2F99270895982FE3
:102E80008091B4058130E1F380B38695869586956F
:102E900080FDF6CF539A9CB981E08093B4050895E4
:102EA0001F93CF93DF93EC011991112359F01A303E
:102EB00019F48DE00E943F17812F0E943F1719914E
:102EC0001123A9F7DF91CF911F9108951092F60574
:102ED0008091F6058093F50508959B01AC01109251
:102EE000F6058091F6058093F5051092B405899A50
:102EF000919A88ED8AB9689413F8220F331F441F02
:102F0000551F1694D1F760E874ED81EE90E00E94B1
:102F1000C421DA01C9010197292F332720BD89B9BE
:102F200086E880BD0895CF93C82F82958F708A3030
:102F300010F4805D01C0895C0E943F178C2F8F7058
:102F40008A3010F4805D01C0895C0E943F17CF91E8
:102F500008958F929F92AF92BF92CF92DF92EF929D
:102F6000FF920F931F93CF93DF93CDB7DEB72297D6
:102F70000FB6F894DEBF0FBECDBF1A8266E770E0D1
:102F800084EC90E00E9456210E942017182F8A306E
:102F900009F41DE080914601882329F01D3019F0C5
:102FA000812F0E943F171D3061F0183051F0113011
:102FB00041F01983BE016F5F7F4F84EC90E00E9467
:102FC0004121183051F484EC90E00E945D2100977B
:102FD00021F0FC01ED53FF4F1082113051F484ECCD
:102FE00090E00E945D21009721F0FC01ED53FF4F1E
:102FF0001082133031F466E770E084EC90E00E94B8
:1030000056211D3009F68091C400882309F431C28D
:1030100080914601882331F08AE00E943F178DE0BD
:103020000E943F1784EC90E00E945D21019779F5A2
:103030008091C400883421F08091C4008F3319F44A
:1030400081E090E018C28091C400823519F484E0D8
:1030500090E011C28091C400893419F482E090E0BC
:103060000AC28091C400863559F48FE794E09F939B
:103070008F930E94012080E090E00F900F90FBC1A1
:103080008091C400843419F485E090E0F4C184ECAC
:1030900090E00E945D21029709F085C068E770E02A
:1030A00084EC90E00E944C21892B09F420C16BE74D
:1030B00070E084EC90E00E944C21009719F410928B
:1030C0004601D9C16EE770E084EC90E00E944C218B
:1030D000892B31F481E0809346018AEF94E0C7C1E7
:1030E00061E870E084EC90E00E944C21892B29F487
:1030F0001092470183E095E0BAC164E870E084EC87
:1031000090E00E944C21892B21F481E080934701BB
:10311000B0C167E870E084EC90E00E944C21009719
:1031200019F410926D01A7C16AE870E084EC90E098
:103130000E944C21892B21F481E080936D0199C17B
:103140006DE870E084EC90E00E944C21892B59F5E9
:1031500080917C0190917D01A0917E01B0917F01D1
:10316000BC01CD010E94A1097B018C018091460127
:10317000882309F47EC11F930F93FF92EF921F9350
:103180000F93FF92EF928FE095E09F938F930E94B1
:1031900001202DB73EB7265F3F4F0FB6F8943EBFD4
:1031A0000FBE2DBF66C184EC90E00E945D210397A5
:1031B00009F048C060E970E084EC90E00E944C2186
:1031C000892BF9F48091AF039091B003A091B103E2
:1031D000B091B2030197A109B10920916201309128
:1031E00063014091640150916501281739074A072E
:1031F0005B0708F07CC0DA01C9010196A11DB11D71
:1032000018C064E970E084EC90E00E944C21892BA6
:10321000C9F48091620190916301A0916401B09121
:1032200065010097A105B10509F461C00197A109E5
:10323000B1098093620190936301A0936401B093FC
:10324000650155C042E050E068E970E084EC90E030
:103250000E946621892B81F487EC90E00E94C01ABD
:10326000882309F006C18AE295E09F938F930E941C
:1032700001200F900F90FDC042E050E06CE970E03B
:1032800084EC90E00E9466216C01892B99F587EC13
:1032900090E00E94911A7B018C018091AF03909184
:1032A000B003A091B103B091B203E816F9060A0782
:1032B0001B07A8F01F930F93FF92EF9288E395E00E
:1032C0009F938F930E940120C6012DB73EB72A5FBE
:1032D0003F4F0FB6F8943EBF0FBE2DBFCCC0E0925B
:1032E0006201F0926301009364011093650186E02E
:1032F00090E0C1C042E050E060EA70E084EC90E011
:103300000E946621892B19F488E090E0B4C042E065
:1033100050E063EA70E084EC90E00E946621892B23
:1033200019F489E090E0A7C043E050E066EA70E05D
:1033300084EC90E00E946621892BA1F487EC90E058
:103340000E941114882309F494C080917201909115
:103350007301A0917401B0917501BC01CD010E946F
:10336000301487C043E050E06AEA70E084EC90E0FB
:103370000E946621892B89F487EC90E00E94911AC3
:103380007B018C0183EB93E00E947A1A43EB53E0BC
:10339000C801B7010E942F156CC043E050E06EEAEF
:1033A00070E084EC90E00E946621892BA9F561E031
:1033B00087EC90E00E94AB12882309F45AC088245D
:1033C0009924540118C0CC24DD248E149F04A00637
:1033D000B10688F4F601EC53FF4F80810E943F173D
:1033E0000894C11CD11CC601AA27BB278E159F05B6
:1033F000A007B10778F368E270E084EC90E00E94E7
:10340000A0117C0100271127E114F1040105110529
:10341000D1F60E94F2132DC043E050E062EB70E061
:1034200084EC90E00E9466218C01892BF1F462E02B
:1034300087EC90E00E94AB12882399F068016CE061
:1034400070E086EB90E00E9485100C9741F40894A0
:10345000C11CD11C30E1C31637E2D30680F30E94B1
:10346000F21384E00E943F1704C083E595E00E94B8
:10347000ED1F80E090E022960FB6F894DEBF0FBEFD
:10348000CDBFDF91CF911F910F91FF90EF90DF9013
:10349000CF90BF90AF909F908F90089589E595E071
:1034A0000E94ED1F89E695E00E94ED1F83E895E0FC
:1034B0000E94ED1F80EA95E00E94ED1F8EEB95E0E3
:1034C0000E94ED1F82EE95E00E94ED1F84E096E0E1
:1034D0000E94ED1F81E296E00E94ED1F8EE396E0D0
:1034E0000E94ED1F87E596E00E94ED1F84E00E9498
:1034F0003F1708950F931F93CF93DF938C01C0E084
:10350000D0E00E942017F801EC0FFD1F8083219668
:1035100082E0C030D807A8F3DF91CF911F910F91BF
:103520000895FC0120E030E040E050E06191662326
:1035300021F1862F80538A30E8F4DA01C9016894BA
:1035400012F8880F991FAA1FBB1F1694D1F7820F7C
:10355000931FA41FB51F280F391F4A1F5B1F862FFB
:103560009927C097AA2797FDA095BA2F280F391F32
:103570004A1F5B1F61916623E1F6CA01B9010895F4
:103580000E941114853019F481E090E0089580E0E4
:1035900090E008950895AF92BF92CF92DF92EF929C
:1035A000FF920F931F93CF93DF9380914D019091E2
:1035B0004E01A0914F01B09150010297A105B105B4
:1035C00018F40E941E1C0CC080914D0190914E0178
:1035D000A0914F01B0915001BC01CD010E945F1C30
:1035E000882309F087C080914D0190914E01A091F0
:1035F0004F01B09150010297A105B10540F48091AF
:103600005D018C3009F487C0803109F484C0A0903A
:103610004D01B0904E01C0904F01D0905001C601B5
:10362000B5010E949C0B7B018C0180918E019091D1
:103630008F01A0919001B0919101E816F9060A0757
:103640001B0710F45701680180918E0190918F0142
:10365000A0919001B0919101E816F9060A071B07A5
:10366000F0F2C601B5010E9443097B018C016F5F36
:103670007F4F8F4F9F4F09F44EC0C0E0D0E083EBE7
:1036800093E0FE01E80FF91F1082219622E0C0307E
:10369000D207B8F3C801B7010E94B60C5B016C01F8
:1036A000C0E0D0E080917A019927C817D90790F43B
:1036B00043EB53E0C601B5010E942F150894A11CED
:1036C000B11CC11CD11C219680917A019927C81781
:1036D000D90770F31092A601C801B7010E94B60C79
:1036E000DC01CB018093AB019093AC01A093AD01C1
:1036F000B093AE0160E070E080E090E00E9443098A
:103700007B018C018FEFE8168FEFF8068FEF08072B
:103710008FEF180719F480E090E014C0E092720176
:10372000F09273010093740110937501109282015D
:103730001092830110928401109285010E94AD1BAA
:1037400081E090E0DF91CF911F910F91FF90EF907A
:10375000DF90CF90BF90AF9008950F931F9380910B
:10376000AB019091AC01A091AD01B091AE0143EBE2
:1037700053E0BC01CD010E94C6148091A601992797
:10378000880F991F82959295907F9827807F982720
:103790008C010D541C4F48E050E06EE971E0C80107
:1037A0000E947421C801089643E050E066E671E08B
:1037B0000E947421F80113861486158620EA3AE9DE
:1037C000268737878AEA9EE2808B918B828B938B48
:1037D000268B378B808F918F80917201909173012E
:1037E000A0917401B0917501CD01AA27BB27848BEC
:1037F000958B8091720190917301828F938F80914C
:10380000820190918301A0918401B0918501848F00
:10381000958FA68FB78F8091AB019091AC01A0914D
:10382000AD01B091AE0143EB53E0BC01CD010E946C
:103830002F1581E090E01F910F910895EF92FF9274
:103840000F931F9320E0EE24FF24870180919201C3
:1038500090919301A0919401B0919501E816F90619
:103860000A071B0728F58091960190919701A09176
:103870009801B09199018E0D9F1DA01FB11FBC0131
:10388000CD010E94B81C282F882391F40894E11CD4
:10389000F11C011D111D8091920190919301A09145
:1038A0009401B0919501E816F9060A071B07D8F2B2
:1038B000822F99271F910F91FF90EF9008959F926B
:1038C000AF92BF92CF92DF92EF92FF920F931F932E
:1038D000CF937B018C01992480918E0190918F016F
:1038E000A0919001B0919101E816F9060A071B0713
:1038F00090F5C801B7010E94B60C5B016C01C0E0F5
:1039000080917A01C81790F4D601C5018C0F911DE2
:10391000A11DB11DBC01CD010E94B81C982E8823A9
:1039200029F4CF5F80917A01C81770F3992099F438
:10393000C801B7010E949C0B7B018C0180918E0114
:1039400090918F01A0919001B0919101E816F90634
:103950000A071B0770F2892D9927CF911F910F91AC
:10396000FF90EF90DF90CF90BF90AF909F90089521
:10397000EF92FF920F931F937B018C0143EB53E077
:103980000E94C61480E090E023EB33E0FC01E20FDC
:10399000F31FE081EE2311F0E53EA9F4E092AB01C4
:1039A000F092AC010093AD011093AE01969587950E
:1039B000929582958F7089279F7089278093A601A1
:1039C00081E090E007C0809642E080309407F0F2FA
:1039D00080E090E01F910F91FF90EF9008954F923B
:1039E0005F926F927F928F929F92AF92BF92CF928F
:1039F000DF92EF92FF920F931F93CF93DF93CDB798
:103A0000DEB72C970FB6F894DEBF0FBECDBF2B01EB
:103A10003C014A01452B49F0AE01475F5F4FBE01B3
:103A20006F5F7F4FC4010E946E1F43EB53E0C301E1
:103A3000B2010E94C614AA24BB2481E08C878501B0
:103A40000D541C4F6801F8018081882319F480E02F
:103A500090E070C1F8018081853E09F45FC1882340
:103A600009F45CC183858F7383878F3009F041C06F
:103A700080916D01882309F451C18114910409F0EA
:103A80004DC18DE796E00E94ED1FFF24F394F601EF
:103A9000EF0DF11D80818F3F11F00E94D61FF2E0E3
:103AA000FF0E89E08F1598F70F2EFEE0FF2EF02D08
:103AB000F601EF0DF11D80818F3F11F00E94D61F9E
:103AC00092E0F90EE8E1EF1598F70F2EFCE1FF2EDA
:103AD000F02DF601EF0DF11D80818F3F11F00E9456
:103AE000D61FF2E0FF0E8EE18F1598F780E896E082
:103AF0007AC08114910409F053C0F801838583FFD3
:103B000003C082E896E009C0F801838584FF03C002
:103B100086E896E002C08AE896E00E94ED1FFF2446
:103B2000F801EF0DF11D80810E94D61FF394F7E09C
:103B3000FF15B0F78EE20E94D61FFF24F801EF0DAB
:103B4000F11D80850E94D61FF39482E08F15B0F797
:103B500080E20E94D61FF801838580FF02C082E5C3
:103B600001C08DE20E94D61FF801838582FF02C04A
:103B700083E501C08DE20E94D61FF801838581FF95
:103B800002C088E401C08DE20E94D61FF80183853F
:103B900085FF02C081E401C08DE20E94D61F19C0DA
:103BA00048E050E0B801CE0101960E946621892BC1
:103BB00011F4F2E0FC87C801089643E050E0BC0134
:103BC000CE0109960E946621892B19F48C858D5FA0
:103BD0008C87F801838583FF09C08114910409F063
:103BE0009DC08EE896E00E94ED1F98C0F801838585
:103BF00084FF29C0848995896C01EE24FF24760115
:103C0000DD24CC24828D938DAA27BB27C80ED91E14
:103C1000EA1EFB1E8114910449F485E996E09F9306
:103C20008F930E9401200F900F9078C0FC85F53093
:103C300009F074C0C0924D01D0924E01E0924F0144
:103C4000F092500168C0F801848995896C01EE24D6
:103C5000FF247601DD24CC24828D938DAA27BB27F7
:103C6000C80ED91EEA1EFB1E81149104B9F4848D7E
:103C7000958DA68DB78DBF93AF939F938F938CE94E
:103C800096E09F938F930E9401208DB79EB7069672
:103C90000FB6F8949EBF0FBE8DBF40C09C85953077
:103CA000E9F548E050E0BE016F5F7F4F8EE991E09B
:103CB0000E94742143E050E0BE01675F7F4F86E6BB
:103CC00091E00E9474214092AB015092AC0160924D
:103CD000AD017092AE01C50196958795929582953A
:103CE0008F7089279F7089278093A601C0927201E7
:103CF000D0927301E0927401F0927501F801848D05
:103D0000958DA68DB78D8093820190938301A093AA
:103D10008401B093850185E090E00CC080E290E0E2
:103D2000A80EB91E90E0A91692E0B90608F485CE57
:103D300081E090E02C960FB6F894DEBF0FBECDBFA9
:103D4000DF91CF911F910F91FF90EF90DF90CF9077
:103D5000BF90AF909F908F907F906F905F904F90AB
:103D600008956F927F929F92AF92BF92CF92DF920F
:103D7000EF92FF920F931F93CF93DC01CB013A0197
:103D80007C018D019924939480918E0190918F01F3
:103D9000A0919001B0919101E816F9060A071B075E
:103DA000A8F5C801B7010E94B60C5B016C01C0E028
:103DB00080917A01C817A0F4D601C5018C0F911D1E
:103DC000A11DB11DA301BC01CD010E94EF1C982EC5
:103DD00081E0981629F4C80F80917A01C81760F322
:103DE00081E0981699F4C801B7010E949C0B7B01F1
:103DF0008C0180918E0190918F01A0919001B091E2
:103E00009101E816F9060A071B0758F2809146014E
:103E1000882319F084E00E943F17892D9927CF91BC
:103E20001F910F91FF90EF90DF90CF90BF90AF90D8
:103E30009F907F906F900895DF92EF92FF920F9383
:103E40001F93CF93DF93EC01DD24D394EE24FF2462
:103E500087018091920190919301A0919401B0917A
:103E60009501E816F9060A071B0738F580919601B7
:103E700090919701A0919801B09199018E0D9F1D8D
:103E8000A01FB11FAE01BC01CD010E94EF1CD82EB6
:103E900081E0D81691F40894E11CF11C011D111D5C
:103EA0008091920190919301A0919401B09195011C
:103EB000E816F9060A071B07C8F280914601882315
:103EC00019F084E00E943F178D2D9927DF91CF9143
:103ED0001F910F91FF90EF90DF900895AF92BF92E6
:103EE000CF92DF92EF92FF920F931F93CF93DF93C6
:103EF0006C015A01EB0110E080E289931F5F1830DA
:103F0000E0F380E2E5018993F50181838983EB0188
:103F1000F60180818E3231F481818E3219F48993D9
:103F2000888339C010E0F601E10FF11D00810E32E7
:103F300051F0002341F0802F99277E0121960E94A5
:103F4000DF21F70180831F5F183020F40E3211F05B
:103F5000002349F7183039F40E3229F0002319F004
:103F6000F60100851F5F0E32B1F4FF24F601E10F68
:103F7000F11D0081002341F0E501CF0DD11D802FFF
:103F800099270E94DF218883F3941F5FF2E0FF15D9
:103F900010F0002359F7DF91CF911F910F91FF90FF
:103FA000EF90DF90CF90BF90AF900895CF93C82F40
:103FB00080914801813041F0CA3019F48DE00E94AF
:103FC0003F178C2F0E943F1780914801882319F0DA
:103FD0008C2F0E949608CF910895CF93DF93EC0128
:103FE000FC0121969491992349F0892F0E94D61FB4
:103FF000FE0121968491982F8823B9F7DF91CF9104
:1040000008952F923F924F925F926F927F928F927C
:104010009F92AF92BF92CF92DF92EF92FF920F9357
:104020001F93CF93DF93CDB7DEB72C970FB6F894DD
:10403000DEBF0FBECDBFE1E2F0E0EC0FFD1FA190AF
:10404000B1901F01F5010894A11CB11C8491853227
:1040500061F0882309F4FCC00E94D61FF501089482
:10406000A11CB11C84918532A1F740E00F2EFAE02B
:104070008F2E9924F02DF5010894A11CB11C849178
:10408000542E442E803311F0803281F4482EF501F5
:104090000894A11CB11C8491982F90539A3030F44D
:1040A000592EF5010894A11CB11C849190E08C3626
:1040B00031F491E0F5010894A11CB11C8491282FE2
:1040C000332723373105E1F0243731053CF423361B
:1040D000310559F02436310559F10FC02537310526
:1040E00069F12837310531F108C0F1012224332468
:1040F000689421F82E0E3F1E80810E94D61FA2CF09
:10410000F10122243324689421F82E0E3F1EC08032
:10411000D180D6018C91882309F494CFF601819146
:104120006F010E94D61FD6018C918823B9F78ACFE0
:1041300041E004C088249924689484F8442351F110
:10414000992361F0F10122243324689422F82E0E81
:104150003F1EE080F180028113810EC0F101222414
:104160003324689421F82E0E3F1E808191817C01BA
:104170000027F7FC0095102F112334F510950095BA
:10418000F094E094E11CF11C011D111D8DE20E94D0
:10419000D61F1AC0992361F0F101222433246894B8
:1041A00022F82E0E3F1EE080F180028113810CC0A8
:1041B000F10122243324689421F82E0E3F1E8081C1
:1041C00091817C01002711270F2EFCE0CF2EDD24EA
:1041D000F02DCC0EDD1E1C86C401AA27BB273C0196
:1041E0004D01C801B701A40193010E94A221262F0D
:1041F000205D2A330CF0295FD6012E936D01C80192
:10420000B701A40193010E94A22179018A015110F2
:104210005A94E114F1040105110519F75A94BFEFFE
:104220005B1639F0F60142926F015A94FFEF5F1668
:10423000C9F7D6018C91882309F404CFF601819146
:104240006F010E94D61FD6018C918823B9F7FACE50
:104250002C960FB6F894DEBF0FBECDBFDF91CF9185
:104260001F910F91FF90EF90DF90CF90BF90AF9094
:104270009F908F907F906F905F904F903F902F9086
:104280000895FB01DC010D900020E9F711970190E2
:104290000D920020E1F70895FB01DC018D91019062
:1042A000801911F40020D1F7990B0895FB01DC016E
:1042B00001900D920020E1F70895FC01019000208B
:1042C000E9F7809590958E0F9F1F0895FB01DC0103
:1042D0004150504030F08D910190801919F4002028
:1042E000B9F7881B990B0895FB01DC014150504040
:1042F00048F001900D920020C9F701C01D92415075
:104300005040E0F70895629FD001739FF001829FB3
:10431000E00DF11D649FE00DF11D929FF00D839F54
:10432000F00D749FF00D659FF00D9927729FB00DF1
:10433000E11DF91F639FB00DE11DF91FBD01CF0104
:1043400011240895A1E21A2EAA1BBB1BFD010DC06A
:10435000AA1FBB1FEE1FFF1FA217B307E407F50735
:1043600020F0A21BB30BE40BF50B661F771F881F11
:10437000991F1A9469F760957095809590959B01A7
:10438000AC01BD01CF01089597FB092E05260ED083
:1043900057FD04D0D7DF0AD0001C38F45095409563
:1043A000309521953F4F4F4F5F4F0895F6F7909509
:1043B0008095709561957F4F8F4F9F4F08958F9394
:1043C00006D08F9109F08F7D089585FD08C0806229
:1043D000992329F481361CF08B370CF40895992722
:0443E000882708958D
:1043E4006175746F747970652E61736D00626F6F9F
:1043F400742E3835340000004453004530004531F4
:10440400004230004231004C30004C310046430041
:1044140044532B0044532D004344200044532000B4
:104424004C2000532000444620005753200052469D
:104434002000464F200048656C6C6F20576F726CEB
:04444400640A000006
:00000001FF
